:100000000C9438000C9453000C9453000C947D0312
:100010000C9489020C9450030C94F6020C94230364
:100020000C945C020C9409020C9453000C94530041
:100030000C9453000C9453000C9453000C945300F4
:100040000C9453000C9453000C9453000C94C9026C
:100050000C9453000000010008004000000100045F
:1000600000000100080020004000800000010004A2
:1000700011241FBECFE5D4E0DEBFCDBF10E0A0E667
:10008000B0E0ECE5F8E002C005900D92A036B107B3
:10009000D9F710E0A0E6B0E001C01D92AC37B1077F
:1000A000E1F70C94AA030C940000039665E070E05D
:1000B0000E94DD03CB01AA27BB2724E0880F991FEC
:1000C000AA1FBB1F2A95D1F720E030E02817390777
:1000D00028F42F5F3F4F28173907D8F30895CF939F
:1000E000C0E08C2F0E94DF00CF5FC830D0F30E94A9
:1000F00080000E948A000E9493007894CF91089516
:1001000082E00E949D0012BE89B7816089BF0E9473
:100110008801089583E00E94A3001DBC1CBC89B720
:10012000846089BF089584E00E94A90014BC89B747
:10013000806489BF0E949C010895982F83B7887FAF
:10014000892B83BF0895982F8EB5887F892B8EBD0C
:100150000895982F85B5887F892B85BD089583B72D
:10016000E82FFF27E770F070EE0FFF1FEC5AFF4FEC
:100170008591949108958EB5E82FFF27E770F07070
:10018000EE0FFF1FEC5AFF4F85919491089585B5AE
:10019000E82FFF27E770F070EE0FFF1FE05AFF4FC8
:1001A000859194910895883040F4E82FFF27EE0F51
:1001B000FF1FE05AFF4F60837183089508958830D0
:1001C00040F4E82FFF27EE0FFF1FE05AFF4F108289
:1001D000118208950895DF92EF92FF920F931F937B
:1001E000CF93DF93EC01D2B6109274001092750099
:1001F00010927600109277000E94AF009C01442775
:10020000552760E074E284EF90E00E941304293BDC
:100210008DE8380786E0480780E05807C0F487E299
:10022000C131D807A0F4CE01AA27BB27BC01CD015C
:100230000E94BE03DC01CB01BC01CD0128EE33E0FE
:1002400040E050E00E94F103FA01E90111C07E0193
:1002500000271127CA01B90128EE33E040E050E041
:100260000E94F103C801B7010E94BE03FC01EB012B
:100270008091740090917500A0917600B091770004
:100280002227382F492F5A2F82B79927AA27BB2711
:10029000282B392B4A2B5B2BCD0DD11DE11DF11DD8
:1002A0002C173D074E075F0758F580917400909119
:1002B0007500A0917600B091770085B78F7485BFE7
:1002C00085B7806485BF889585B78F7B85BF809112
:1002D000740090917500A0917600B091770022276C
:1002E000382F492F5A2F82B79927AA27BB27282BA7
:1002F000392B4A2B5B2B2C173D074E075F07A8F2C3
:10030000DF91CF911F910F91FF90EF90DF900895B3
:10031000109270001092710010927200109273008F
:1003200008958091700090917100A0917200B09139
:100330007300BC01CD0108951092780010927900ED
:1003400010927A0010927B0008958091780090912D
:100350007900A0917A00B0917B00BC01CD01089595
:10036000893031F48FB582608FBD8FB58E7F0AC022
:100370008A3019F48FB5826002C08FB58D7F8FBD32
:100380008FB581608FBD1BBC1ABC19BC18BC089509
:100390009C018FB58E7F8FBD8FB582608FBD8EB56E
:1003A00088608EBD8EB580618EBD37BD26BD1BBCFD
:1003B0001ABC19BC18BC08958FB58D7F8FBD8FB541
:1003C0008E7F8FBD0E94F5010E94FC0108958FB5BC
:1003D00080688FBD8FB58F7B8FBD08958FB580628C
:1003E0008FBD8FB58F7E8FBD08958FB58F778FBDF1
:1003F0008FB58F7B8FBD08958FB58F7D8FBD8FB5E6
:100400008F7E8FBD08959BBD8ABD089599BD88BD1F
:1004100008951F920F920FB60F9211242F933F93BE
:100420004F935F936F937F938F939F93AF93BF93FC
:10043000EF93FF938091700090917100A0917200F2
:10044000B09173000196A11DB11D8093700090932F
:100450007100A0937200B09373008091740090912A
:100460007500A0917600B09177000196A11DB11D95
:100470008093740090937500A0937600B0937700FA
:100480008091600090916100892B29F0E0916000DB
:10049000F09161000995FF91EF91BF91AF919F910C
:1004A0008F917F916F915F914F913F912F910F901D
:1004B0000FBE0F901F9018951F920F920FB60F92BC
:1004C00011242F933F934F935F936F937F938F9359
:1004D0009F93AF93BF93EF93FF93809162009091AE
:1004E0006300892B29F0E0916200F0916300099587
:1004F000FF91EF91BF91AF919F918F917F916F91FC
:100500005F914F913F912F910F900FBE0F901F90D1
:1005100018951F920F920FB60F9211242F933F93AD
:100520004F935F936F937F938F939F93AF93BF93FB
:10053000EF93FF938091780090917900A0917A00D9
:10054000B0917B000196A11DB11D8093780090931E
:100550007900A0937A00B0937B0080916A0090911B
:100560006B00892B29F0E0916A00F0916B000995EE
:10057000FF91EF91BF91AF919F918F917F916F917B
:100580005F914F913F912F910F900FBE0F901F9051
:1005900018951F920F920FB60F9211242F933F932D
:1005A0004F935F936F937F938F939F93AF93BF937B
:1005B000EF93FF9380916E0090916F00892B29F04B
:1005C000E0916E00F0916F000995FF91EF91BF915E
:1005D000AF919F918F917F916F915F914F913F91DB
:1005E0002F910F900FBE0F901F9018951F920F9292
:1005F0000FB60F9211242F933F934F935F936F93F6
:100600007F938F939F93AF93BF93EF93FF938091CB
:10061000640090916500892B29F0E0916400F091CD
:1006200065000995FF91EF91BF91AF919F918F91D7
:100630007F916F915F914F913F912F910F900FBEDE
:100640000F901F9018951F920F920FB60F921124C2
:100650002F933F934F935F936F937F938F939F93CA
:10066000AF93BF93EF93FF938091660090916700E3
:10067000892B29F0E0916600F09167000995FF91C0
:10068000EF91BF91AF919F918F917F916F915F910A
:100690004F913F912F910F900FBE0F901F90189583
:1006A0001F920F920FB60F9211242F933F934F93E7
:1006B0005F936F937F938F939F93AF93BF93EF93CA
:1006C000FF938091680090916900892B29F0E09157
:1006D0006800F09169000995FF91EF91BF91AF918A
:1006E0009F918F917F916F915F914F913F912F914A
:1006F0000F900FBE0F901F9018951F920F920FB67C
:100700000F9211242F933F934F935F936F937F9397
:100710008F939F93AF93BF93EF93FF9380916C0060
:1007200090916D00892B29F0E0916C00F0916D00A3
:100730000995FF91EF91BF91AF919F918F917F911B
:100740006F915F914F913F912F910F900FBE0F903E
:100750001F901895CFE5D4E0DEBFCDBF8FE081BB01
:1007600082BB0E946F00909884EF91E00E94EB00A2
:10077000909A84EF91E00E94EB00F5CF629FD00148
:10078000739FF001829FE00DF11D649FE00DF11D4C
:10079000929FF00D839FF00D749FF00D659FF00DFB
:1007A0009927729FB00DE11DF91F639FB00DE11DE8
:1007B000F91FBD01CF0111240895AA1BBB1B51E1F4
:1007C00007C0AA1FBB1FA617B70710F0A61BB70BC1
:1007D000881F991F5A95A9F780959095BC01CD0166
:1007E0000895A1E21A2EAA1BBB1BFD010DC0AA1F72
:1007F000BB1FEE1FFF1FA217B307E407F50720F08A
:10080000A21BB30BE40BF50B661F771F881F991F04
:100810001A9469F760957095809590959B01AC014D
:10082000BD01CF01089597FB092E05260ED057FD77
:1008300004D0D7DF0AD0001C38F45095409530958D
:1008400021953F4F4F4F5F4F0895F6F79095809554
:0C085000709561957F4F8F4F9F4F08956A
:00000001FF
